:01659B0022DD
:10244A007584008537D28538D37584018539D2855C
:10245A003AD3E4F538F537300006853B37853C3802
:10246A0030010CE537253DF537E538353EF538308E
:10247A000210E548852EF0A42537F537E5F0353802
:10248A00F538300310E50A8531F0A42537F537E52C
:10249A00F03538F538300410E5118530F0A42537C9
:1024AA00F537E5F03538F538E4F53AF539300810FE
:1024BA00853B39853C3AE53CC39535400385353A39
:1024CA00300916E53EC39534400385353EE5392586
:1024DA003DF539E53A353EF53A300A10E548852E9C
:1024EA00F0A42539F539E5F0353AF53A300B10E51F
:1024FA000A8531F0A42539F539E5F0353AF53A304F
:10250A000C10E5118530F0A42539F539E5F0353A96
:10251A00F53A300D10E518852FF0A42539F539E57F
:10252A00F0353AF53A300E10E52C8533F0A425390A
:10253A00F539E5F0353AF53A300F10E52D8532F0E8
:10254A00A42539F539E5F0353AF53AE53AC3953631
:10255A00400385363A2290264C302D0312258230CC
:07256A002E03122592303010
:10257100031225F9302F031225B530310312260934
:1025810022E50B2509F50BE50C3508F50C93F50A49
:1025910022E512250EF512E513350DF51393C3133C
:1025A100F8E5142510F514E515350FF51593C3134A
:1025B10028F51122103908203A3C303D238026D2DB
:1025C1003A203B0E303C2FC23AC23DC23B756B00F4
:1025D1008024203C21C23AD23DD23B756B0080164B
:1025E10090274C8003902794E56B93F52C056BE5C0
:1025F1006BB44802D23A2222E5192517F519E51ADA
:102601003516F51A93F51822103E08203F3C30424A
:10261100238026D23F20400E30412FC23FC242C20A
:1026210040756C008024204121C23FD242D24075C6
:102631006C0080169027FC80039027DCE56C93F5F5
:102641002D056CE56CB44802D23F227F8285888CCF
:102651008F9295989B9EA1A4A7AAADB0B3B6B9BB22
:10266100BEC1C3C6C9CBCED0D3D5D7D9DCDEE0E25B
:10267100E4E6E7E9EBEDEEF0F1F2F4F5F6F7F8F95F
:10268100FAFBFCFCFDFDFEFEFEFEFEFEFEFEFEFE76
:10269100FDFDFCFCFBFAFAF9F8F7F6F4F3F2F0EFC2
:1026A100EDECEAE8E7E5E3E1DFDDDBD8D6D4D1CF35
:1026B100CDCAC8C5C2C0BDBAB7B4B2AFACA9A6A392
:1026C100A09D9A9794908D8A8784817E7A77747180
:1026D1006E6B6865625F5C595653504D4A47444280
:1026E1003F3C393734322F2D2A282624211F1D1B28
:1026F1001918161412110F0E0C0B0A0807060504FF
:1027010004030202010100000000000000000000BB
:1027110001010202030405060708090A0B0D0E1048
:1027210011131516181A1C1E20222427292B2E30AE
:102731003335383A3D404245484B4E515456595C29
:10274100606366696C6F7275787B7FFEFEFEFEFDCD
:10275100FCFCFBFAF8F7F6F4F3F1EFEDEBE9E7E453
:10276100E2DFDCDAD7D4D0CDCAC6C3BFBCB8B4B0BF
:10277100ACA8A39F9B96928D89847F7A75706B66B6
:10278100615C57514C47413C37312C26211B1610B7
:102791000B050000050B10161C21272C32373D427A
:1027A100484D53585D62686D72777C81858A8F943C
:1027B100989DA1A5AAAEB2B6BABEC1C5C8CCCFD2AA
:1027C100D5D8DBDEE1E3E6E8EBEDEFF1F2F4F6F785
:1027D100F8F9FBFBFCFDFEFEFEFEFE000C192633A4
:1027E1003F4C5864707B86919CA6AFB8C1C9D1D8C3
:1027F100DEE4EAEFF3F6F9FCFDFEFEFEFDFCFAF77E
:10280100F4F0EBE6E0DAD4CCC5BCB4ABA1978D8390
:0B281100786D61554A3D3125180C0020
:1043CD00D2F4C2F5C2F675840F85F0C8122BD474E1
:1043DD000312441C122BC8740312441C122BAB1273
:1043ED002BAB740312441C122BAB740212441C121F
:1043FD002BAB74281244887406124488740E124430
:10440D00887401124488122BC8748012448822C00B
:10441D0000A2E092F3A2E192F2A2E292F1A2E39263
:10442D00F0D2F475840F85F0C8C2F47830D8FE85CB
:10443D00F0C87830D8FED00022C00075840FA2E4F9
:10444D0092F3A2E592F2A2E692F1A2E792F0D2F4F3
:10445D0085F0C8C2F47830D8FE85F0C87830D8FE23
:10446D00D00022EF75840FD2F5C2F685F0C8124444
:10447D0046122BAB12441C122BAB2275840FC2F5C6
:10448D00C2F685F0C8124446122BAB12441C122BF7
:10449D00AB22EF14A2E492E6C2E4D2E712448822E2
:1044AD00740F12448822740D124488227F01124425
:1044BD009F78107F20124470D8F9227F1112449FEB
:1044CD0078107F20124470D8F9227F0112449F7812
:0944DD00207F20124470D8F9225E
:104E7200758400D2C2C2C6D2C6C2C4D2C5C2C330B1
:104E8200C3FD74A0F5C2C2C5C2C330C3FD8EC2C287
:104E9200C330C3FD8FC2C2C330C3FD8DC2C2C33093
:104EA200C3FDD2C4C2C320C4FD122BC82275840024
:104EB200C2C3D2C530C3FD74A0F5C2C2C5C2C330DD
:104EC200C3FD8EC2C2C330C3FD8FC2C2C330C3FD95
:104ED200C2C4D2C5C2C330C3FD74A1F5C2C2C5C229
:104EE200C330C3FDC2C2C2C330C3FD85C207D2C430
:064EF200C2C320C4FD2232
:08000300023199000000000029
:08000B0002319D00000000001D
:080013000233050000000000AB
:0C001B00C28FB2A1320000000000000003
:09002300320000000000000000A2
:08002B000231A00000000000FA
:08003300320000000000000093
:0A003B003200000000000000000089
:0900430032000000000000000082
:08004B0032000000000000007B
:08005300320000000000000073
:08005B0002320E00000000005B
:08006300320000000000000063
:08006B00023226000000000033
:080073000231A10000000000B1
:08007B00023308000000000040
:08008300023208000000000039
:08008B0032000000000000003B
:1000930002332A00000000000000000000000000FE
:1000A3003275FF0775FFDE75FFAD75840F75E107C8
:1000B30075E20475E34475840F75A43575A5097558
:1000C300A6FF75A7FF759CFF759D00759E00759F24
:1000D300F075D8FF75E8FF75F80F75AD0F758401DE
:1000E30075893075888F75840275893075888F7529
:1000F300840F758A80758C67780874FF0000000090
:100103000000000000000000D5E0F1D8EDE58C30E0
:10011300E7FB759701758A0043890475840075B7F9
:100123001075840F438901758D01758F01758E02DA
:100133007480D5E0FD438902E58930E4FB759702BD
:1001430075840075D10775840075BB0175BA007598
:10015300BCF075C70075C60075C5FF75C4FF75E8AB
:100163008175840275BB0475BA0075BCF175C60050
:1001730075C4FF75E88875840075D484758401752A
:10018300D484758400C2F8759A47759D1A43F8099B
:1001930075870075840075B90075A90075910075A0
:1001A300985075840175981075840075C04075C3A7
:1001B3000075CFC9758400758E1075892075880503
:1001C300758400758A00758B70758CF4758D70431A
:1001D300885075840075C90075CA0075CB0075CC4D
:1001E3000075CD0075840175C91875CA8075CBFB80
:1001F30075CDFB75CC80D2CA75840275C91875CAD2
:10020300A675CBAF75CDAF75CCA6D2CA7584007574
:10021300EF0075A88575B80075E6A475E71775F640
:100223000075F7019000007F007E20E4F0A3DFFC5F
:02023300DEFAF1
:10023500752EFF752FFF7530FF7531FF7532FF7510
:1002450033FF7534FF7535FF7536FF751D0A751E4D
:050255000A751F0622DE
:1031990002281C32C28D3232C007C006C005C004E5
:1031A900C0E0C083C082C0D0C000C0F0C001C2CF9F
:1031B900B232203220151BE51B7009751B0A758474
:1031C900017588AF151CE51C7009751C60758402B2
:1031D9007588AF800E153FE53F7008753F0475840B
:1031E90000D28B758400D2ECD001D0F0D000D0D0C1
:1031F900D082D083D0E0D004D005D006D00732C227
:10320900CF02053D32C0E0C0D0E54060021540E57F
:10321900436002154375888FD0D0D0E032C007C013
:10322900E0C0D0C000C084202A1375840F30DF2588
:10323900E5E8540FF549D22A754AC88018154AE5B8
:103249004A7006E549D2E7F54975840F20DF06C2C1
:103259002AD229D251202C1475840F30F828E5E898
:1032690054F0C4F54BD22C754CC8801A154CE54C5A
:103279007006E54BD2E7F54B75840F20F808C22C90
:10328900D22BD250D237E54160021541E55D60028B
:10329900155D7880E6600116151DE51D7051751DD7
:1032A9000AE54260021542E54460021544E55960A9
:1032B900021559E55A6002155A788CE6600116E53F
:0932C9005760021557E558600238
:1032D2001558E57760021577151EE51E7018751EE4
:1032E2000AE55C6002155C151FE51F7009751F0673
:1032F200E55B6002155BD084C28DD000D0D0D0E0F7
:10330200D0073202025AC0D020280DD22885BF3EF3
:1033120085BE3D75BB01800BC22885BF3C85BE3B87
:1033220075BB00C2EDD0D032C0E0C0D0E54DB400D4
:103332000A054D85BE4875BB07803DB4010A054D9F
:1033420085BE4575BB048030B4020A054D85BE4872
:1033520075BB068023B4030A054D85BE4675BB04C2
:103362008016B4040A054D85BE4875BB05800975F3
:0F3372004D0085BE4775BB04C2EDD0D0D0E03210
:102B3B0075840FD2FD2275840FC2FD2275840FD2CE
:102B4B00FC2275840FC2FC2275840FD2FED2452263
:102B5B0075840FC245C2FE22C29322D29322758482
:102B6B000FA2FA2275840FA2F92275840FA2DD221F
:102B7B0075840FA2DE22A2922275840FA2DA22752F
:102B8B00840FA2DB2275840FA2D82275840FA2D9E1
:102B9B0022000000000000000000000000000022E6
:102BAB00C000C001790478B4D8FED9FAD001D000A6
:102BBB0022C0007814122BABD8FBD00022C0E075DA
:102BCB004005E54070FCD0E022C0E075400FE540C9
:102BDB0070FCD0E022C0E0754064E54070FCD0E0B2
:102BEB0022A42582F582E58335F0F58322B40A0011
:102BFB0022C0E0C3997001D3D0E022B50601225068
:102C0B0007B5070122400122D322EF75F06484241B
:102C1B00309000A1F0E5F0A375F00A842430F0A306
:102C2B00E5F02430F022EF75F0648424309000A19D
:072C3B00F0E5F0A375F00ABB
:102C4200842430F0A3E5F02430F09000A1E0B43009
:102C52000B7420F0A3E0B430037420F02290000D36
:102C6200E0540FFFA3E0B420028019540FCF75F097
:102C72000AA42FFFA3E0B420028009540FCF75F0FD
:102C82000AA42FFF22C006C005C00490000DE05424
:102C92000FFFFEA3E0B42003C3802C540FFDCF75B9
:102CA200F00AA42FFFA3E0B42003C3801A540FFC40
:102CB200EE75F064A420D20EFEED75F00AA42E404B
:102CC200052C40028001D3D004D005D0062275F035
:102CD2006484F6E5F00875F00A84F608A6F0082286
:102CE200C0017900E6B4FF028027F908E6B4FF03C9
:102CF200C38022E975F00AA426F908E6B4FF03C3EB
:102D02008013E975F00AA420D207C3264003F98094
:102D120004D3D00122E9D00122E675F00AA40826E4
:102D2200227850EE122CD0754E00754F00785290DA
:042D32002D7C790873
:102D3600EF134007A3A3A3A3A3801CC0E0C000C059
:102D460001C37905E49336D4A2E4540FF6A318D947
:102D5600F3D001D000D0E0D9D8E54E600C754F090C
:102D6600755009755109755209854F4E85504F8525
:102D7600515085525122060502000002010500004D
:102D86000402000100080400020006090004000213
:0E2D96000901080004080306010806070203ED
:105BA4002A2A3132333435362A2A2A2A31323334F6
:105BB40035302A2A44313233343536373839302AAD
:105BC4002341424320202056455253494F4E203111
:105BD4002E31202020204D554C54492D4445434F0F
:045BE40044455220C2
:104CB20030501DC250E54B540F905BB8939000CE1C
:104CC200F0788C7632302115125FB7125E29800D92
:104CD200788CE670089000BAF09000CBF030513A30
:104CE200C251E549540F905BB8939000CDF07557CF
:104CF200329000BFE004F030450320200620450634
:104D0200302203125DEE30450320200320450312BA
:104D12005F82204511126021800CE55770089000D7
:104D2200BBF09000CAF0304C1630231F7558321277
:104D320065959000BEEFF0C24C125E64025FECE536
:0C4D42005870089000BCF09000CCF022EB
:105F82009000BBE0FF04F0EF905BA493FF9000CD84
:105F9200E0FEEF6E6011EEB42A089000BB7401F0CF
:105FA2008005E49000BBF09000BBE0B40A06E4F088
:055FB200D248D252228A
:105FB7009000BAE0FF04F0EF905BA493FF9000CE4F
:105FC700E0FEEF6E6011EEB42A089000BA7401F09B
:105FD7008005E49000BAF09000BAE0B40A06E4F055
:055FE700D247D2522256
:105FEC009000BCE0FF04F0EF905BA493FF9000BE28
:105FFC00E0FEEF6E6011EEB42A089000BC7401F064
:10600C008005E49000BCF09000BCE0B40A06E4F01B
:05601C00D249D252221E
:105DEE009000CAE0FF04F074C12FF582E43400F590
:105DFE0083E0FF9000CDE0FEEF6E6011EEB423085D
:105E0E009000CA7401F08005E49000CAF09000CAB8
:0B5E1E00E0B40906E4F0D248D24622AE
:105E29009000CBE0FF04F074C12FF582E43400F553
:105E390083E0FF9000CEE0FEEF6E6011EEB4230820
:105E49009000CB7401F08005E49000CBF09000CB7A
:0B5E5900E0B40906E4F0D247D2462274
:105E64009000CCE0FF04F074C12FF582E43400F517
:105E740083E0FF9000BEE0FEEF6E6011EEB42308F5
:105E84009000CC7401F08005E49000CCF09000CC3C
:0B5E9400E0B40906E4F0D249D2462237
:106021009000BDE0FF04F0EF905BAE93FF9000CDD8
:10603100E0FEEF6E6011EEB42A089000BD7401F02D
:106041008005E49000BDF09000BDE0B40A04E4F0E6
:03605100D2532205
:1061AA009000C17423F0A3F0E4FF74AD2FF582E4EC
:1061BA003400F583E0FE74C32FF582E43400F583DE
:0C61CA00EEF00FBF06E49000C97423F053
:0161D60022A6
:106087001243CD1244B91244C87F0112449F7BFFCB
:106097007A5B79D81260F07BFF7A5B79C81261214D
:1060A70075421EE54270FCE49000BFF01244B9024D
:0260B70044C8DB
:036595007F012261
:1033810075540012339C50FB2275540012342550A1
:10339100FB227554001233DC50FB22758400E55486
:1033A10075F003A49033A9730234410234500234FE
:1033B1006E02345702347A02348102348902345065
:1033C1000234970234570234A70234B00234410266
:1033D10034500234BE0234570234CA758400E554B5
:1033E10075F003A49033E97302344102345002347E
:1033F1006E02345702347A0234810234410234506D
:1034010002346E02345702347A02348102347A0271
:1034110034810234890234500234CC0234570234EC
:10342100A70234CA758400E55475F003A4903432C0
:10343100730234410234500234BE0234570234CA9A
:10344100C2FA1234DC1234DC759B000554C32230FD
:10345100F9020554C32230F912E59A20E7FB123430
:10346100DCD2FA1234DC1234DC0554C322C2FA1263
:1034710034DC759B040554C32275431E0554C322D5
:10348100E54370020554C322C2FA1234DC1234FD42
:10349100F59B0554C322C2FA1234DC12350C4407E1
:1034A100F59B0554C3221234EEF5440554C322752D
:1034B100840F30DE04E54470020554C322C2FA12BF
:1034C10034DC759B080554C322D322C2FA1234DCC2
:0934D10012350C4405F59B05546D
:1034DA00C3220000000000000000000000000000FD
:1034EA00000000229034F5E55593225A5A5A5A5A46
:1034FA00FAFAFA903504E555932200B45AE12D8779
:10350A007ADB903513E55593220000000000008015
:01351A008030
:100D130043544353532036332E30202020202020A9
:100D230043544353532036372E3020202020202095
:100D330043544353532036392E342020202020207F
:100D430043544353532037312E3920202020202071
:100D530043544353532037342E3420202020202063
:100D630043544353532037372E3020202020202054
:100D730043544353532037392E372020202020203B
:100D830043544353532038322E3520202020202033
:100D930043544353532038352E3420202020202021
:100DA30043544353532038382E352020202020200D
:100DB30043544353532039312E3520202020202003
:100DC30043544353532039342E38202020202020ED
:100DD30043544353532039372E34202020202020DE
:100DE3004354435353203130302E302020202020D1
:100DF3004354435353203130332E352020202020B9
:100E03004354435353203130372E322020202020A7
:100E13004354435353203131302E39202020202096
:100E23004354435353203131342E38202020202083
:100E33004354435353203131382E3820202020206F
:100E43004354435353203132332E3020202020206B
:100E53004354435353203132372E33202020202054
:100E63004354435353203133312E38202020202044
:100E73004354435353203133362E35202020202032
:100E83004354435353203134312E33202020202028
:100E93004354435353203134362E32202020202014
:100EA3004354435353203135312E34202020202006
:100EB3004354435353203135362E372020202020EE
:100EC3004354435353203135392E382020202020DA
:100ED3004354435353203136322E322020202020D6
:100EE3004354435353203136352E352020202020C0
:100EF3004354435353203136372E392020202020AA
:100F03004354435353203137312E332020202020A4
:100F13004354435353203137332E3820202020208D
:100F23004354435353203137372E3320202020207E
:100F33004354435353203137392E39202020202066
:100F43004354435353203138332E3520202020205F
:100F53004354435353203138362E3220202020204F
:100F63004354435353203138392E39202020202035
:100F73004354435353203139322E3820202020202C
:100F83004354435353203139362E3620202020201A
:100F93004354435353203139392E35202020202008
:100FA3004354435353203230332E35202020202006
:100FB3004354435353203230362E352020202020F3
:100FC3004354435353203231302E372020202020E6
:100FD3004354435353203231382E312020202020D4
:100FE3004354435353203232352E372020202020C0
:100FF3004354435353203232392E312020202020B2
:101003004354435353203233332E362020202020A1
:101013004354435353203234312E38202020202090
:101023004354435353203235302E33202020202085
:101033004354435353203235342E31202020202073
:10104300202020202020202020202020202020209D
:101053004443532030303620494E5620303231201D
:101063004443532030303720494E56203231342008
:101073004443532030313520494E562031343120FA
:101083004443532030313720494E562030353020E9
:101093004443532030323120494E562030303620DD
:1010A3004443532030323320494E562030343720C6
:1010B3004443532030323520494E562032343420B5
:1010C3004443532030323620494E562034363420A0
:1010D3004443532030333120494E56203632372093
:1010E3004443532030333220494E5620303531208B
:1010F3004443532030333620494E56203137322073
:101103004443532030343320494E56203434352061
:101113004443532030343720494E56203032332055
:101123004443532030353020494E56203031372048
:101133004443532030353120494E5620303332203A
:101143004443532030353320494E56203435322022
:101153004443532030353420494E56203431332014
:101163004443532030363520494E56203237312000
:101173004443532030373120494E562033303620F4
:101183004443532030373220494E562032343520E1
:101193004443532030373320494E562035303620D0
:1011A3004443532030373420494E562031373420BE
:1011B3004443532031313420494E562037313220B5
:1011C3004443532031313520494E562031353220A6
:1011D3004443532031313620494E5620373534208D
:1011E3004443532031323220494E56203232352087
:1011F3004443532031323520494E5620333635206F
:101203004443532031333120494E56203336342062
:101213004443532031333220494E5620353436204F
:101223004443532031333420494E56203232332045
:101233004443532031343120494E56203031352038
:101243004443532031343320494E56203431322025
:101253004443532031343520494E5620323734200D
:101263004443532031353220494E56203131352005
:101273004443532031353520494E562037333120EE
:101283004443532031353620494E562032363520DB
:101293004443532031363220494E562035303320D3
:1012A3004443532031363520494E562032353120C0
:1012B3004443532031373220494E562030333620B1
:1012C3004443532031373420494E5620303734209D
:1012D3004443532032303520494E56203236332092
:1012E3004443532032313220494E56203335362081
:1012F3004443532032313420494E56203030372076
:101303004443532032323320494E56203133342064
:101313004443532032323520494E56203132322055
:101323004443532032323620494E56203431312043
:101333004443532032343320494E56203335312031
:101343004443532032343420494E56203032352022
:101353004443532032343520494E5620303732200F
:101363004443532032343620494E562035323320FD
:101373004443532032353120494E562031363520EF
:101383004443532032353220494E562034363220DE
:101393004443532032353520494E562034343620C9
:1013A3004443532032363120494E562037333220BE
:1013B3004443532032363320494E562032303520B1
:1013C3004443532032363520494E5620313536209A
:1013D3004443532032363620494E56203435342088
:1013E3004443532032373120494E5620303635207E
:1013F3004443532032373420494E5620313435206C
:101403004443532033303620494E56203037312061
:101413004443532033313120494E5620363634204D
:101423004443532033313520494E56203432332040
:101433004443532033323520494E5620353236202B
:101443004443532033333120494E5620343635201C
:101453004443532033333220494E5620343535200C
:101463004443532033343320494E562035333220FE
:101473004443532033343620494E562036313220EC
:101483004443532033353120494E562032343320E0
:101493004443532033353620494E562032313220CF
:1014A3004443532033363420494E562031333120C0
:1014B3004443532033363520494E562031323520AC
:1014C3004443532033373120494E56203733342099
:1014D3004443532034313120494E56203232362092
:1014E3004443532034313220494E56203134332083
:1014F3004443532034313320494E56203035342071
:101503004443532034323320494E5620333135205F
:101513004443532034333120494E5620373233204D
:101523004443532034333220494E5620353136203C
:101533004443532034343520494E5620303433202D
:101543004443532034343620494E56203235352017
:101553004443532034353220494E5620303533200E
:101563004443532034353420494E562032363620F6
:101573004443532034353520494E562033333220EB
:101583004443532034363220494E562032353220DC
:101593004443532034363420494E562030323620CB
:1015A3004443532034363520494E562033333120BB
:1015B3004443532034363620494E562036363220A3
:1015C3004443532035303320494E562031363220A0
:1015D3004443532035303620494E5620303733208C
:1015E3004443532035313620494E5620343332207C
:1015F3004443532035323320494E5620323436206B
:101603004443532035323620494E56203332352059
:101613004443532035333220494E5620333433204C
:101623004443532035343620494E5620313332203B
:101633004443532035363520494E56203730332026
:101643004443532036303620494E5620363331201A
:101653004443532036313220494E5620333436200A
:101663004443532036323420494E562036333220F9
:101673004443532036323720494E562030333120ED
:101683004443532036333120494E562036303620DA
:101693004443532036333220494E562036323420C9
:1016A3004443532036353420494E562037343320B3
:1016B3004443532036363220494E562034363620A2
:1016C3004443532036363420494E5620333131209B
:1016D3004443532037303320494E56203536352086
:1016E3004443532037313220494E56203131342080
:1016F3004443532037323320494E5620343331206C
:101703004443532037333120494E56203135352059
:101713004443532037333220494E5620323631204A
:101723004443532037333420494E56203337312036
:101733004443532037343320494E56203635342022
:101743004443532037353420494E56203131362017
:102DA40075840F1200A41260879000D9E4F0A3E4A4
:102DB400F09000D7E4F0A3E4F0789276007890766F
:102DC400007894760078977600788D7600788E7601
:102DD40000788F7600124CB230534C12659BC2536C
:102DE40080451260541262791261AA9000B9E4F02D
:102DF400C247C248C249802F802DC25212630312B7
:102E04005F131262791261AA9000B9E4F0C247C25A
:102E140048C249757F00E57FC3941E5007122BE01A
:102E2400057F80F2126087122885125B5CE577705B
:102E3400061244B975771E12291D9000D5EFF030A3
:102E440036659000D5E0FF9000D3E0FEEEB50705AF
:102E5400788D06800E9000D5E0FF9000D3EFF078D7
:102E64008D7601788DE6FFEFC394034038205A3500
:102E74009000D3E0FF7895A6077895E6FF7E10EFE3
:102E84008EF0A4FFAEF074132FF9740D3EFA7BFF9D
:102E94001260F0D25A9000D3E0FF7895A6077577B8
:102EA4000F788D7600C23630334E9000D4E0FFEFB9
:102EB400B55E05788F06800A9000D4E55EF0788FC1
:102EC4007601788FE6FFEFC39403402A205B27AF97
:102ED4005E7E10EF8EF0A4FFAEF074532FF97410E1
:102EE4003EFA7BFF1260F0D25B75770A788F76002A
:102EF400C236788D7600C23330566090008DE0FF84
:102F04009000D1E0FEEEB5071390008EE0FF900034
:102F1400D2E0FEEEB50705788E068018788E76012D
:102F240090008DE0FF9000D1EFF090008EE0FF90D4
:102F340000D2EFF0788EE6FFEFC39403401B205CD1
:102F440018124D4EC236788D7600C233788F7600D3
:102F5400D25C75770A788E7600C2567894E6FFEFD5
:102F640070147890E6FFEF700D7892E6FFEF70062C
:102F7400205D031257B6305A06205D031254D33035
:102F84005B06205D031250EF305C06205D03124B9C
:0D2F940075205D03022E2B124A0F022E2B1A
:012FA100220D
:10025A00C0D0C000C001C083C082C0E0C0F0A2927A
:10026A0020A001B37864E233F208E233F208E23301
:10027A00F208E233F208E233F208E233F208E23338
:10028A00F208E233F208E233F208E233F208E23328
:10029A00F208E233F208E233F208E233F208E23318
:1002AA00F208E233F208E233F208E233F208E23308
:1002BA00F208E233F208E233F208E233F208E233F8
:1002CA00F208E233F208E233F208E233F208E233E8
:1002DA00F208E233F208E233F208E233F208E233D8
:1002EA00F208E233F208E233F208E233F208E233C8
:1002FA00F208E233F208E233F208E233F208E233B8
:10030A00F208E233F29006C3788BE218936028E28F
:10031A0018937023E21893601EE218937019E2187A
:10032A00936014E21893600FE21893700AE218932C
:10033A007005E2189360030204EF755F00E21893F8
:10034A001392545003755F38752300E21893139281
:10035A001C5003635F1CE2189313921B5003635FE4
:10036A000EE2189313921A5003635F46E21893132E
:10037A0092195003635F23E218931392188523603E
:10038A005003635F51752300E2189313921C5003C4
:10039A00635F68E2189313921B5003635F75E21858
:1003AA009313921A5003635F7AE2189313921950C7
:1003BA0003635F3DE2189313921885236150036328
:1003CA005F1F752300E2189313921F5003635F4F58
:1003DA00E2189313921E5003635F26E21893139256
:1003EA001D5003635F52E2189313921C5003635F1C
:1003FA0029E2189313921B5003635F15E2189313B3
:10040A00921A5003635F0BE2189313921950036315
:10041A005F45E218931392188523625003635F6263
:10042A00E2189313921C5003635F31E218931392FC
:10043A001B5003635F19E2189313921A5003635F08
:10044A000DE218931392195003635F07E21893138E
:10045A0092188523635003635F43752300E2189360
:10046A0013921EE2189313921DE2189313921CE240
:10047A00189313921BE2189313921AE21893139289
:10048A0019E21893139218852364C257E564655FCD
:10049A006035D25723F8900C1493F9900C13E89313
:1004AA006025B40104B254801EB40205E86260807B
:0D04BA0016B40305E86261800EB40405E885
:1004C70062628006B40521E86263A25492559000E7
:1004D7008CE560F090008DE561F090008EE562F0AC
:1004E70090008FE563F0D256120501D0F0D0E0D02E
:1004F70082D083D001D000D0D0327882E660363007
:1005070031337881E6D5E02D76087882167887E64C
:10051700A2E0304301B39241D23EA2E07883E613D2
:10052700F67884E613F67885E613F67886E613F60A
:100537007887E613F622C0D0C000C001C083C0820E
:10054700C0E0C0F0C258A292205801B3784CE21321
:10055700F208E213F208E213F208E213F208E213D8
:10056700F208E213F208E213F208E213F208E213C8
:10057700F208E213F208E213F208E213F208E213B8
:10058700F208E213F208E213F208E213F208E213A8
:04059700F208E21371
:10059B00F208E213F208E213F208E213F208E21394
:1005AB00F208E213F29006C3784CE2089313921709
:1005BB00E20893139216E20893139215E208931331
:1005CB009214E20893139213E20893139212E20827
:1005DB0093139211E20893139210852265E208930C
:1005EB00139217E20893139216E20893139215E2F3
:1005FB000893139214E20893139213E20893139245
:10060B0012E20893139211E208931392108522665B
:10061B00E20893139217E20893139216E2089313CE
:10062B009215E20893139214E20893139213E208C3
:10063B0093139212E20893139211C210852267E56D
:10064B0065900A13856622301602058393602D147C
:10065B00F875F003A49008C42582F582E5F0358384
:10066B00F583E493F9A3E4939007C3656793C96596
:10067B00669329B401005004885ED233120699D0D8
:10068B00F0D0E0D082D083D001D000D0D032302F48
:10069B00267888E6D5E0207608788BE6A2E1304410
:1006AB0001B3923CD239A2E17889E613F6788AE657
:1006BB0013F6788BE613F622000000000000000012
:1006CB00000000000000000000000000000000001F
:1006DB00000000000000000100000000000000000E
:1006EB0000000000000000010000000000000001FD
:1006FB0000000001000101010000000000000000EB
:10070B0000000000000000010000000000000001DC
:10071B0000000001000101010000000000000001C9
:10072B0000000001000101010000000100010101B6
:10073B0000010101010101010000000000000000A7
:10074B00000000000000000100000000000000019C
:10075B000000000100010101000000000000000189
:10076B000000000100010101000000010001010176
:10077B000001010101010101000000000000000166
:10078B000000000100010101000000010001010156
:10079B000001010101010101000000010001010143
:1007AB000001010101010101000101010101010130
:1007BB00010101010101010100010102010202031A
:1007CB0001020203020303040102020302030304F6
:1007DB0002030303030304050102020302030304E0
:1007EB0002030304030404050203030403040405C6
:1007FB0003040404040505060102020302030304B7
:10080B0002030303030404050203030403030405A7
:10081B00030404050405050602030304030404058D
:10082B000304040504050506030404050405050675
:10083B00040505060506060701020203020303046D
:10084B000203030403040405020303040304040565
:10085B00030404050405050602030304030404054D
:10086B000304040504050506030404050405050635
:10087B000405050605060607020303040304040525
:10088B000304040504050506030404050405050615
:10089B0004050506050606070304040504050506FD
:1008AB0004050506050606070405050605060607E5
:1008BB000506060706070708FDD00C73700E3CF003
:1008CB001AAF101E7F9022EC7026D6F02ACBB02CDC
:1008DB00A3F032BEB03417D03CB6D0461FB04E7723
:1008EB00F050F950526AB056DE9058BA306ACF3099
:1008FB0072D270745CD076E8F0786BD098E5709A11
:10090B00F8309CBB50A40F70AA7A70B26730B45DFC
:10091B00B0B8FCB0C26F50C655D0CA3D90D489B0A8
:10092B00DA94F0DCD790E463B0EA0BF0F43170F8B2
:10093B00DD310AB571148FF118D1D126EB512AF69E
:10094B00112C8B71463F5148B1F14AACB14CC4F1FB
:10095B0052D9B1546D915A2EF162BD116687916ACD
:10096B009AD16CF29172D5517819F18C71B192D8F0
:10097B00D19A32D1AA47D1B25A91B452F1C675313C
:10098B00CC1D71D2A951DCD0B1E85E11EA2B11F26A
:10099B00EED212F392147D3216973226D8B232C5AC
:1009AB00F234F7124AEA524C9F5254A5D2582B728A
:1009BB005A7552644FD268C1726ADC326C78D28637
:0D09CB005F128C83729C4EB2A66972AC1C48
:1009D80072B433D2CC18F2EABB330CCE33141EB344
:1009E8002803F32EE51332F8533498735848F36408
:1009F80072736845738617B3947313A63C93B22138
:100A0800D3B41B53B829B3C641F3D8000000000083
:100A180000000000000000000000000000000000CE
:100A280000006A000000000000620D0000000000E5
:100A3800000000006F0048000000000000000000F7
:100A4800000000000000006C220000000000000010
:100A58000000000000000000005B00000000000033
:100A680000000000004100001E4759000000260059
:100A780000001D0000100000350000003D006B0064
:100A880043000000000000004B00050000000000CB
:100A980000003800230000000000000000000000F3
:100AA80000004C00000000000000000000000000F2
:100AB80000000000000000320000040000000000F8
:100AC8000000000000126000370A0000000000006B
:100AD800000000000000080000611346000000004C
:100AE8000000254D340000572911000000000000C7
:100AF800640000000000000000000000003A4A0006
:100B0800002E4F190000001F0000000000006300C5
:100B1800000000000000270000001B00000000008B
:100B280000000B5F3C006E5D440000006D0000009B
:100B3800000000000000530000360000283F5E005F
:100B480000000000000000030000300070000000FA
:100B580069004067000000000000550000420000E6
:100B68002100000000000015000000000000000047
:100B7800000000005C001700000020000068020070
:100B880054000E58001C00000000000000005A002D
:100B98000000000000002F0000002B0000000024CF
:100BA8000000006600390000000051000000090044
:100BB8005200000045000000000000003100000065
:100BC8002A0C000000001A00000000005600003344
:100BD8004E00000000000000000000002C1400007F
:100BE8003B07003E0000000000000000000000007D
:100BF8001800001600502D060049000000000000F3
:100C0800000000650F000000010000000000000067
:100C180000060000000600060005020600060006A1
:100C28000004040600050402080600000006000689
:100C3800000600060004080600060006000508066F
:100C48000006000210060006000301000006000668
:100C58000002020600060004400600060004100612
:100C6800000600060006000600060006000510063D
:100C78000006000600060006000600010106000640
:100C88000006000600030206000600000006000633
:100C9800000501060004020204060006000600061C
:100CA8000006000600060006000480060002010493
:100CB80020060006000600060006000600060006DC
:100CC80000060006000600060006000600060004EE
:100CD80001060006000600060006000310060006CE
:100CE80000060006000600060006000600060006CC
:100CF80000060006000308060006000600060003BA
:0B0D08000406000600060006000600BE
:10281C00C0D0C0E0C084758400C2CA85CC6E85CDA2
:10282C006D75CC0075CD00D2CA10CF41203443E574
:10283C0068B4000A856D6F856E7005688032B401CE
:10284C000A856D71856E7205688025B4020A856DE6
:10285C0073856E7405688018B40312856D75856E6A
:10286C0076D234756800D084D0E0D0D03275680050
:10287C00C234D084D0E0D0D032C0D0C0E0C000C0D0
:10288C0001C002C003C004C005C006C00730346CD0
:10289C00AA70AB6FAE02AF03EEC4035407FEEFC4D5
:1028AC0003FF54F84EFEEF5407FFC3E5729AFCE5A4
:1028BC00719BFD50066304FF6305FFC3EC9EED9F07
:1028CC005038C3E5749AFCE5739BFD50066304FF16
:1028DC006305FFC3EC9EED9F5020C3E5769AFCE5A3
:1028EC00759BFD50066304FF6305FFC3EC9EED9FD3
:1028FC005008856F6A857069D235C234D007D0060E
:10290C00D005D004D003D002D001D000D0E0D0D07C
:10291C002230352B902A3BE56A93FF90296F2323B5
:0A292C002582F582E5833400F5836F
:1029360012294E400E0F12294E40080F12294E4002
:10294600028002D236C23522E493F9A3E493FAA3B5
:10295600E493FBA3E493FCA3C3E5699AE56A995063
:1029660007C3EC9569EB956A22EA25DD89DD89D3F3
:1029760024D324CBD2CBD2C4DBC4DBBE39BE39B719
:10298600CAB7CAB18EB18EAB87AB87A59CA59CA0F2
:1029960000A0009A969A9695D895D891E591E58DDE
:1029A600858D8588AF88AF840C840C7F9A7F9A7B4F
:1029B600497B49771B771B730F730F6F276F276B45
:1029C600576B5767AB67AB642C642C60C660C65DFB
:1029D600795D795AFE5AFE5970597057E257E25698
:1029E60061566154E754E7537453745207520750C3
:1029F600A050A04F404F404DE64DE64C934C934BB4
:102A0600414B4149F549F548B548B54776477646BD
:102A16003E463E45084508432A432A40E440E43FF3
:102A2600533F533E3E3E3E3C943C943A863A86396A
:102A360018391838053232323232323232323232C4
:102A46003232323232323232323232323232323260
:102A56003232323232323232323232323232323250
:102A66003232323232323232323232323232313142
:102A760030302F2E2D2D2D2C2C2B2A292928272698
:102A86002525242323222120201F1E1E1D1C1C1B3E
:102A96001A1A1A1A191919181818171717171616AD
:102AA60016161515151514141414131313131212E0
:102AB60012121111111110101010100F0F0F0F0F0D
:102AC6000E0E0E0E0E0D0D0D0C0C0C0C0B0B0B0B37
:102AD6000B0B0A0A0A0A0A0909090909090808085A
:102AE6000808080707070707070606060606060674
:102AF600050505050505040404040404040303038D
:102B060003030303020202020202020101010101A0
:102B160001010101010101010100000000000000A6
:102B2600000000000000000000000000000000009F
:052B360000000000009A
:104D4E007F0112449F7F4C1244707F541244707F37
:104D5E00521244707F201244702055047F3080021E
:104D6E007F311244707F2012447090008DE0784E97
:104D7E00122CD8784E8607430730124470088607E7
:104D8E0043073012447075072012447090008EE075
:104D9E00784E122CD0784E86074307301244700896
:104DAE0086074307301244700886074307301244C3
:104DBE007075072012447090008CE0784E122CD83B
:104DCE00784E860743073012447008860743073033
:0A4DDE001244707507201244702281
:1063DA0044313233343536373839302A234142434F
:105B5C00303744E54B540FFFEF9063DA93FF90001E
:105B6C00D9E475F001124847ADF0FC74DB2DF582D9
:105B7C0074003CF583EFF0124DE8C2379000D9E089
:105B8C00FEA3E0FFEFB4200CEEB403089000D9E4C0
:085B9C00F0A3E4F0755B0222A6
:1057B6009000D7E0FEA3E0FF9000D9E0FCA3E0FD57
:1057C600EDB50706ECB5060222229000D7E475F087
:1057D60001124847AFF0FE74DB2FF58274003EF5E8
:1057E60083E0FF7898A6079000D7E0FEA3E0FFEFDE
:1057F600B4200CEEB403089000D7E4F0A3E4F0D292
:025806005D2221
:104DE800E54B540FFFEF9063DA93FF8F7D9000C07F
:104DF800E0FFEFD3940F50269000C0E0FFEF24119E
:104E0800FF12449F9000C0E0FF04F074912FF582D8
:104E1800E43400F583E57DF0AF7D124470227F1104
:104E280012449F757E00E57EC3940F5031AF7E74A7
:104E3800922FF582E43400F583E0FFAE7E74912E64
:104E4800F582E43400F583EFF0AF7E74912FF5829C
:104E5800E43400F583E0FF124470057E80C89000BA
:094E6800A0E57DF0AF7D1244705D
:014E7100221E
:104A0F007584009000D6E0FFEF700F758400C29997
:104A1F007599549000D6E004F0229000D6E0FFEF95
:104A2F00B40112209903024AC4C29975993A9000B1
:104A3F00D6E004F0229000D6E0FFEFB4020F3099D9
:104A4F0074C2997599209000D6E004F0229000D698
:104A5F00E0FFEFB4031230995CC2997898E6FF8FAC
:104A6F00999000D6E004F0229000D6E0FFEFB40456
:104A7F000F309941C29975990D9000D6E004F0223C
:104A8F009000D6E0FFEFB4050F309929C2997599C0
:104A9F000A9000D6E004F0229000D6E0FFEFB406B3
:104AAF000D309911C2999000D6E4F0C25D229000AA
:064ABF00D6E4F0C25D2206
:10206E00303036203032313030372032313430316A
:10207E003520313431303137203035303032312067
:10208E00303036303233203034373032352032343F
:10209E003430323620343634303331203632373025
:1020AE00333220303531303336203137323034331D
:1020BE002034343530343720303233303530203020
:1020CE0031373035312030333230353320343532FC
:1020DE0030353420343133303635203237313037E5
:1020EE0031203330363037322032343530373320EA
:1020FE0035303630373420313734313134203731C2
:10210E0032313135203135323131362037353431B7
:10211E0032322032323531323520333635313331A9
:10212E0020333634313332203534363133342032A5
:10213E003233313431203031353134332034313291
:10214E003134352032373431353220313135313575
:10215E00352037333131353620323635313632206F
:10216E003530333136352032353131373220303358
:10217E003631373420303734323035203236333240
:10218E00313220333536323134203030373232333B
:10219E00203133343232352031323232323620343D
:1021AE00313132343320333531323434203032351C
:1021BE003234352030373232343620353233323500
:1021CE003120313635323532203436323235352003
:1021DE0034343632363120373332323633203230E1
:1021EE0035323635203135363236362034353432C6
:1021FE0037312030363532373420313435333036BE
:10220E0020303731333131203636343331352034C6
:10221E00323333323520353236333331203436359E
:10222E00333332203435353334332035333233348F
:10223E003620363132333531203234333335362091
:10224E003231323336342031333133363520313278
:10225E00353337312037333434313120323236345E
:10226E00313220313433343133203035343432335B
:10227E002033313534333120373233343332203555
:10228E00313634343520303433343436203235352B
:10229E003435322030353334353420323636343519
:1022AE003520333332343632203235323436342020
:1022BE0030323634363520333331343636203636F6
:1022CE0032353033203136323530362030373335F3
:1022DE0031362034333235323320323436353236DD
:1022EE0020333235353332203334333534362031E2
:1022FE0033323536352037303336303620363331BB
:10230E0036313220333436363234203633323632AA
:10231E0037203033313633312036303636333220B3
:10232E00363234363534203734333636322034367E
:10233E003636363420333131373033203536353773
:10234E003132203131343732332034333137333177
:10235E00203135353733322032363137333420336E
:10236E003731373433203635343735342031313642
:10237E002036333020363730203639342037313955
:10238E00203734342037373020373937203832353C
:10239E002038353420383835203931352039343825
:1023AE002039373431303030313033353130373207
:1023BE0031313039313134383131383831323330DE
:1023CE0031323733313331383133363531343133CD
:1023DE0031343632313531343135363731353938AD
:1023EE0031363232313635353136373931373133A0
:1023FE00313733383137373331373939313833357F
:10240E003138363231383939313932383139363668
:10241E003139393532303335323036353231303775
:10242E003231383132323537323239313233333666
:0C243E003234313832353033323534312D
:1054D3007892E6B41200505D9054E2F828287302E3
:1054E300551802552A02551B02552A02551E02550C
:1054F3002A02552002552A02552202552A02552412
:1055030002552A02552702552A02552C02552A0212
:10551300553202553502648F02644180078005804D
:105523000302651D0261D7800302652702649B02A3
:065533006531126417222D
:0C648F00E4F584C29975994378920622C6
:0C649B00E4F584309905C299789206223D
:0D644100E4F58475993A7893F67892062276
:1061D700E4F5847893E606FF7895E625E025E02444
:1061E7007EF582E43423F583E5822FF582E4358357
:0A61F700F583E493F59978920622EF
:0A651D00E4F58475992E78920622A9
:0A652700E4F58475990D78920622C0
:0A653100E4F58475990A78920622B9
:0E641700E4F584309907C2997892F6C25A22B1
:1050EF007890E6B41600506C9050FEF828287302A2
:1050FF00514002515502514302515502514602513E
:10510F005502514802515502514A02515502514C14
:10511F0002515502514E0251550251500251550242
:10512F00515202515502515702515502515D0251D0
:10513F00600264A702644E800A80088006800480A3
:10514F00028000026201800302653B0264B30265C4
:05515F00451264252249
:0C64A700E4F584C29975994478900622AF
:0C64B300E4F584309905C2997890062227
:0D644E00E4F58475993A7891F6789006226D
:10620100E4F5847891E606FF75F007E55EA4246E57
:10621100F582E5F03420F583E5822FF582E43583BC
:0A622100F583E493F59978900622C6
:0A653B00E4F58475990D78900622AE
:0A654500E4F58475990A78900622A7
:0E642500E4F584309907C2997890F6C25B22A4
:104B75007894E6B41E004003024C14904B87F82845
:104B85002873024BE1024C06024BE4024C06024B31
:104B9500E7024C06024BEA024C06024BEC024C06BD
:104BA500024BEF024C06024BF2024C06024BF4029A
:104BB5004C06024BF7024C06024BFA024C06024B1E
:104BC500FD024C06024C00024C06024C03024C0648
:104BD500024C08024C06024C0E024C110264BF0244
:104BE500654F0263C8801102633502645B80090268
:104BF500634A02646802647502655902635F026470
:104C05008280030265630264CB02656D1264332200
:0C64BF00E4F584C29975994C789406228B
:0C64CB00E4F584309905C299789406220B
:0A654F00E4F58475993A7894062269
:1063C800E4F58430550575993180037599307894D2
:0263D80006229B
:0A655900E4F5847599207894062279
:1063350090008DE0FF122C15E4F5849000A2E0F5A5
:05634500997894062286
:0D645B00E4F5849000A3E0F5997894062202
:10634A0090008EE0FF122C15E4F5849000A1E0F590
:05635A00997894062271
:0D646800E4F5849000A2E0F59978940622F6
:0D647500E4F5849000A3E0F59978940622E8
:10635F0090008CE0FF122C15E4F5849000A2E0F57C
:05636F0099789406225C
:0D648200E4F5849000A3E0F59978940622DB
:0A656300E4F58475990D7894062282
:0A656D00E4F58475990A789406227B
:0E643300E4F584309907C2997894F6C25C2291
:1017530044313233343536373839302A2341424322
:1017630044AAA3C1C2C3C4D7ABA8A92A23414243F5
:10177300010101010101010101000000000000005D
:101783000000000000000000000000000000000056
:101793000000000000000000000000000000000046
:1017A3000000000000000000000000000000000036
:1017B3000000000000000000000000000000000026
:1017C3000000000000000000000001010101010110
:1017D3000101010000000000000000000000000003
:1017E30000000000000000000000000000000000F6
:1017F30000000000000000000000000000000000E6
:1018030000000000000000000000000000000000D5
:1018130000000000000000000000000000000000C5
:1018230000000000010101010101010101000000AC
:1018330000000000000000000000000000000000A5
:101843000000000000000000000000000000000095
:101853000000000000000000000000000000000085
:101863000000000000000000000000000000000075
:1018730000000000000000000000000000006E06F1
:10188300001102061501016E100611030115010175
:101893006401161104051501010000000000000099
:1018A3000000000000000000000000000000000035
:1018B3000000000000000000000000000000000025
:1018C3000000000000000000000000000000000015
:1018D30000000000000000000101010101010101FD
:1018E30001000000000000000000000000000000F4
:1018F30000000000000000000000000000000000E5
:1019030000000000000000000000000000000000D4
:1019130000000000000000000000000000000000C4
:1019230000000000000000000000000000000000B4
:10193300000001010101010101010100000000009B
:101943000000000000000000000000000000000094
:101953000000000000000000000000000000000084
:101963000000000000000000000000000000000074
:101973000000000000000000000000000000000064
:1019830000000000000000000000000020202020D4
:101993002020202020202020202020202020202044
:1019A3002020202020202020202020202020202034
:1019B3002020202020202020202020202020202024
:1019C3002020202020202020202020202020202014
:1019D3002020202020202020202020202020202004
:1019E30020202020202020202020202020202020F4
:1019F30020202020202020202020202020202020E4
:101A030020202020202020202020202020202020D3
:101A130020202020202020202020202020202020C3
:101A23002020202020202020202020202020204192
:101A33004E49204E554D4245522020202020202043
:101A4300414E49204E414D452020202020415558EC
:101A53002052454C41592056414C494420202020D6
:101A63002020202020202020313D454E20202020F2
:101A7300202020202020202020414E4920202020EB
:101A83002020202020202020202020202020202053
:101A93002020202020202020202020202020202043
:101AA300474C4F42414C20202020202020435443C8
:101AB300535320434F4445202020202020204443DB
:101AC3005320434F44452020202020204C545220B3
:101AD30052455045415445522020202020414E4933
:101AE30020504152414D4554455253205350454592
:101AF300442043414C4C494E47202020205054431E
:101B0300204E554D424552202020202020564F493B
:101B13004345204D455353414745532020564F4994
:101B2300434520504C41594241434B202020494ECC
:101B330056414C49442054595045202020204F55AC
:101B430054204F462052414E4745202020494C4CBB
:101B53004547414C2056414C554520204D55535443
:101B63002046494C4C204649454C44202020494CB2
:101B73004C4547414C20434F444520202044415489
:101B83004120414343455054454420204C494E4550
:101B9300204E554D4245523A202020205553455260
:101BA3002050524F4752414D4D494E475553455290
:101BB3002049443A2020202020202020564F49430A
:101BC30045205245434F5244494E472020494C4CEF
:101BD3004547414C20454E545259202020494C4CF6
:101BE3004547414C2047414E472020202020204399
:101BF3004F4D504C45544544202020203633303639
:101C03003730363934373139373434373730373979
:101C13003738323538353438383539313539343861
:101C2300393734313030313033313037313130318D
:101C33003134313138313233313237313331313379
:101C43003631343131343631353131353631353958
:101C53003136323136353136373137313137333149
:101C6300373731373931383331383631383931391B
:101C7300323139363139393230333230363231302C
:101C8300323138323235323239323333323431321F
:101C9300353032353430303630303730313530311D
:101CA300373032313032333032353032363033310F
:101CB30030333230333630343330343730353030FC
:101CC30035313035333035343036353037313037E0
:101CD30032303733303734313134313135313136D5
:101CE30031323231323531333131333231333431D0
:101CF30034313134333134353135323135353135B1
:101D03003631363231363531373231373432303598
:101D13003231323231343232333232353232363298
:101D23003433323434323435323436323531323579
:101D33003232353532363132363332363532363663
:101D4300323731323734333036333131333135335F
:101D5300323533333133333233343333343633354B
:101D63003133353633363433363533373134313135
:101D73003431323431333432333433313433323433
:101D83003435343436343532343534343535343609
:101D930032343634343635343636353033353036FE
:101DA30035313635323335323635333235343635EF
:101DB30036353630363631323632343632373633DC
:101DC30031363332363534363632363634373033CD
:101DD30037313237323337333137333237333437BE
:101DE30034333735344142434445464748494A4BE7
:101DF3004C4D4E4F505152535455565758595A61A2
:101E030062636465666768696A6B6C6D6E6F707137
:101E130072737475767778797A3031323334353634
:101E2300373839607E21402324255E262A28295FFE
:101E33002D2B3D7B7D5B5D7C3A3B3C3E2C2E3F2F27
:101E430020202020202020202064010011021115D1
:101E5300010164020011031115010164040011045E
:101E6300111501016408001105111501017806011E
:101E7300110601190101820207110712150063827D
:101E830002081108121500638202091109131500D3
:101E93006382030A110A151500FF82030B110B1548
:101EA3001500FF641000110C1115051982020C11A5
:101EB3000D1415016382020D110E141500638202C5
:101EC3000E110F1415006382020F11101315016315
:101ED30020202020202020202020202020202020FF
:101EE30020202020202020202020202020202020EF
:101EF3002054454C434F2050524F4752414D2020D0
:101F030020524144494F2050524F4752414D2020C7
:101F13002050484F4E452050524F4752414D2020AC
:101F230020434F4D50552050524F4752414D202092
:101F3300202041434345535320434F444520202011
:101F4300205455524E204F4E2044454C4159202099
:101F5300205455524E204F46462044454C4159206B
:101F63005455524E2041524F554E4420444C592013
:101F730044544D462054454C434F204C4556454C04
:101F830044544D4620524144494F204C4556454CFC
:101F930041555820524C5920494E56414C494420F2
:101FA30020494E56414C49442054494D4552202026
:101FB300202056414C49442054494D45522020206D
:101FC3002020444953504C41592054494D45202029
:101FD300204348415241435445522054494D4520E2
:101FE300202020202020202020202020313D454E6D
:101FF30020202020202020202020203130204D535D
:1020030020202020202020202020313030204D533C
:102013002020202020202020202020202053454342
:102023002020202020202020202020524154494FCE
:102033000F3132333435360A6314FF320505050A8E
:10204300000000000000000000000000000000008D
:1020530000000000202020202020202020202020FD
:0B206300202020202020202020200032
:10605400755B64E4900000F030470B304624125D19
:1060640070122FA280F530480B304616125DAF1225
:106074002FA280F530490B30460812351B122FA28F
:0360840080F52282
:102FA200E55B7012900000E0D394004009C247C272
:102FB20048C249C24622900000E012486930B90076
:102FC20030BC0130BF0230C20330C50430C7053007
:102FD200C90630CB0730CE0830D10A30D40B30D7F7
:102FE2000F30DA1030DD1430E01530E31930E61A14
:102FF20030E91B30EC1E30EF1F30F22330F5243065
:10300200F82830FB2930FE2D31012E31042F3107F3
:1030120030310A32310D33310F343112353115640A
:10302200311865311B66311E6731216E31236F31D4
:103032002570316771312778312979312B7A3167DF
:103042007B312D82312F8331318431338531368C7E
:1030520031398D313B8E313D8F314096314397313D
:103062004598314799314AA0314DA13150A2315290
:10307200A33155AA3157AB315AAC315CAD315FB493
:103082003162B53165B63167B73169BE316CBF3176
:103092006FC03172C13167C23178F0317BF1317E5C
:1030A200F23181FA3184FB3187FC318AFD318DFEA8
:1030B2003190FF000031930263EA0262E4025CB1E4
:1030C20002622B800480028000025A350236890295
:1030D20060B9023AAE025808023BFC02585A023D5D
:1030E2004A025CF20255F602428202599C023E9862
:1030F200025A7F023FE6025AC902413402617C024F
:103102005EDA025C6F125B13025652800002532C8D
:10311200025C2C0258AC025BE8025F4C0256AC80A7
:10312200468032804B804080228045800780268006
:103132003F0259E902488F801C80350258FD024F38
:103142007D8008802B025D31024AC502524E8020EA
:1031520002494F80120250768016023955024FFA08
:1031620002539A800B800C02516402594D024C1595
:10317200025E9F0257600262520254030263F90226
:10318200570602659C02659D02659E0252BD02655C
:073192009FE4900000F02211
:0F63EA00E4900002F0755B64900000E004F02284
:1062E4001244B91244C87BFF7A1B799F1260F07F75
:0F62F4001112449FC24DC24A900000E004F022F4
:105CB100304A3D900001E0FFC24ABF2A0790000030
:105CC100E004F022EF642370277F231244709000D8
:105CD10002E004F0E0C394034010C247C248C24945
:105CE100C246E4900000F00260879000007402F068
:015CF1002290
:10622B007BFF7A1B799F1260F01244C87F111244D6
:10623B009F1264D7E490003CF07F2A124470C24D49
:07624B00900000E004F022C6
:105A3500304A46900001E0F578C24AE578642A606C
:105A450038AF781264085022AF7812447090003C49
:105A5500E02403F582E43400F583E578F090003C1A
:105A6500E004F0900000E004F0227BFF7A1B79CF80
:095A75001260F090000074FAF0D8
:015A7E002205
:10368900204A030237F3900001E0FFC24ABF2A072C
:103699009000007403F022EF642360030237E41200
:1036A9004470900004E064397077A3E06439707164
:1036B900A3E06439706BD24E900003E0FFB4310887
:1036C900E4900036F0023753EFB43208E490003743
:1036D900F0023766EFB43302803E900003E0FFB496
:1036E9003408E4900038F0023794EFB43508E490D8
:1036F9000039F00237AAEFB43608E490003AF00234
:1037090037C0EFB437028010900003E0B43802806C
:1037190007900003E0B4390B7BFF7A1B79DF02378E
:10372900EAC24E900003E0FFB43016A3E0B43011B2
:10373900A3E0B4300CA3E0B43007900000740AF0A1
:1037490022EFB4310C1255995007900000740FF014
:1037590022900003E0B4320C125539500790000052
:103769007414F022900003E0B43311A3E0B4300CD8
:103779001262C350079000007419F022900003E010
:10378900B4340FA3E0B4300A126374900000741EBD
:10379900F022900003E0B4350FA3E0B4300A1263BD
:1037A900899000007423F022900003E0B4360FA33F
:1037B900E0B4300A12639E9000007428F022900051
:1037C90003E0B43716A3E0B43011A3E0B4300CA37E
:1037D900E0B43007900000742DF0227BFF7A1B794A
:0A37E900CF1260F090000074FAF0B7
:0137F30022B3
:1060B90090003B740BF090003C7407F0E4900049A9
:1060C900F090004AF090004BF07BFF7A1A799F120A
:1060D90060F012611B7F1E12449F9000007432F021
:0160E9002294
:103AAE001251D9D39000A7E0940A9000A6E094009A
:103ABE00400A1260EA90000074FAF0229000A6E02C
:103ACE00FEA3E0FF901E4C75F00912485DEE75F0F6
:103ADE0009A42583F583E493900040F0901E4D7564
:103AEE00F009EF12485DEE75F009A42583F583E425
:103AFE0093900041F09000A6A3E0901E4E75F00941
:103B0E0012485DEE75F009A42583F583E4939000C9
:103B1E0042F0901E4F75F009EF12485DEE75F009F8
:103B2E00A42583F583E493900043F09000A6A3E0D0
:103B3E00901E5075F00912485DEE75F009A42583AC
:103B4E00F583E493FD900044F0901E5175F009EF5B
:103B5E0012485DEE75F009A42583F583E493900079
:103B6E0045F09000A6A3E0901E5275F00912485D34
:103B7E00EE75F009A42583F583E493900046F0904A
:103B8E001E5375F009EF12485DEE75F009A42583FA
:103B9E00F583E493900047F09000A6A3E0901E54A6
:103BAE0075F00912485DEE75F009A42583F583E4DE
:103BBE0093900048F0ED6015900044E075F010A46D
:103BCE0024D3F9741E35F0FA7BFF1260F090004595
:103BDE00E0FF601175F010A424D3F9741E35F0FACD
:0E3BEE007BFF126121900040E0900000F02269
:1058080090003B7410F090003C7407F0E49000495D
:10581800F090004AF0900036E090004BF07BFF7A61
:105828001A79AF1260F012611B7F0D12449F90002D
:1058380004E0FF124470900005E0FF1244709000ED
:1058480006E0FF1244707F1E12449F9000007432DD
:02585800F0223C
:103BFC001251D9D39000A7E094009000A6E0940055
:103C0C00400A1260EA90000074FAF0229000A6E0DC
:103C1C00FEA3E0FF90177375F00912485DEE75F086
:103C2C0009A42583F583E493900040F090177475F4
:103C3C00F009EF12485DEE75F009A42583F583E4D5
:103C4C0093900041F09000A6A3E090177575F009D1
:103C5C0012485DEE75F009A42583F583E49390007A
:103C6C0042F090177675F009EF12485DEE75F00989
:103C7C00A42583F583E493900043F09000A6A3E081
:103C8C0090177775F00912485DEE75F009A425833D
:103C9C00F583E493FD900044F090177875F009EFEC
:103CAC0012485DEE75F009A42583F583E49390002A
:103CBC0045F09000A6A3E090177975F00912485DC5
:103CCC00EE75F009A42583F583E493900046F090FB
:103CDC00177A75F009EF12485DEE75F009A425838B
:103CEC00F583E493900047F09000A6A3E090177B37
:103CFC0075F00912485DEE75F009A42583F583E48F
:103D0C0093900048F0ED6015900044E075F010A41D
:103D1C00248FF9741935F0FA7BFF1260F09000458E
:103D2C00E0FF601175F010A4248FF9741935F0FAC6
:0E3D3C007BFF126121900040E0900000F02219
:10585A0090003B7415F090003C7407F0E490004906
:10586A00F090004AF0900037E090004BF07BFF7A0E
:10587A001A79BF1260F012611B7F0C12449F9000CC
:10588A0004E0FF124470900005E0FF12447090009B
:10589A0006E0FF1244707F1E12449F90000074328B
:0258AA00F022EA
:103D4A001251D9D39000A7E094009000A6E0940005
:103D5A00400A1260EA90000074FAF0229000A6E08D
:103D6A00FEA3E0FF9017CD75F00912485DEE75F0DD
:103D7A0009A42583F583E493900040F09017CE754B
:103D8A00F009EF12485DEE75F009A42583F583E486
:103D9A0093900041F09000A6A3E09017CF75F00928
:103DAA0012485DEE75F009A42583F583E49390002B
:103DBA0042F09017D075F009EF12485DEE75F009E0
:103DCA00A42583F583E493900043F09000A6A3E032
:103DDA009017D175F00912485DEE75F009A4258394
:103DEA00F583E493FD900044F09017D275F009EF43
:103DFA0012485DEE75F009A42583F583E4939000DB
:103E0A0045F09000A6A3E09017D375F00912485D1B
:103E1A00EE75F009A42583F583E493900046F090AB
:103E2A0017D475F009EF12485DEE75F009A42583E1
:103E3A00F583E493900047F09000A6A3E09017D58D
:103E4A0075F00912485DEE75F009A42583F583E43F
:103E5A0093900048F0ED6015900044E075F010A4CE
:103E6A0024AFF9741935F0FA7BFF1260F09000451F
:103E7A00E0FF601175F010A424AFF9741935F0FA57
:0E3E8A007BFF126121900040E0900000F022CA
:105CF2007BFF7A1A79CF1260F07BFF7A1B79AF12A1
:105D020061217F0E12449F900005E0FF12447090C3
:105D12000006E0FF1244707F1A12449F90003B7409
:0F5D22001AF090003C7404F09000007432F022EC
:1055F600304F079000007403F02212611B7F1E12C9
:10560600449F12546C9000A8E0FEA3E0FFD39400E0
:10561600EE9400402DEF94FBEE9400502590003B55
:10562600741BF090003C7407F0E4900049F0900081
:105636004AF0900035E01490004BF0900000743270
:0C564600F0221260EA90000074FAF022DA
:10428200D39000A7E094009000A6E09400400A12A8
:1042920060EA90000074FAF0229000A6E0FEA3E02B
:1042A200FF90182775F00912485DEE75F009A425F4
:1042B20083F583E493900040F090182875F009EF9D
:1042C20012485DEE75F009A42583F583E49390000E
:1042D20041F09000A6A3E090182975F00912485DFC
:1042E200EE75F009A42583F583E493900042F090E3
:1042F200182A75F009EF12485DEE75F009A42583BE
:10430200F583E493900043F09000A6A3E090182B6D
:1043120075F00912485DEE75F009A42583F583E472
:1043220093FD900044F090182C75F009EF12485D4F
:10433200EE75F009A42583F583E493900045F0908F
:1043420000A6A3E090182D75F00912485DEE75F0F5
:1043520009A42583F583E493900046F090182E7506
:10436200F009EF12485DEE75F009A42583F583E4A8
:1043720093900047F09000A6A3E090182F75F009E3
:1043820012485DEE75F009A42583F583E49390004D
:1043920048F0ED6015900044E075F010A424CFF9C8
:1043A200741935F0FA7BFF1260F0900045E0FF606F
:1043B2001175F010A424CFF9741935F0FA7BFF12AD
:0B43C2006121900040E0900000F0221C
:10599C0090003B741FF090003C7407F09000497429
:1059AC0064F090004A7417F0900038E090004BF0CF
:1059BC007BFF7A1A79DF1260F012611B7F0F1244A1
:1059CC009F900005E0FF124470900006E0FF124427
:0D59DC00707F1E12449F9000007432F02274
:103E98001251D9D39000A7E094039000A6E09400B3
:103EA800400A1260EA90000074FAF0229000A6E03E
:103EB800FEA3E0FF90188175F00912485DEE75F0D9
:103EC80009A42583F583E493900040F09018827547
:103ED800F009EF12485DEE75F009A42583F583E437
:103EE80093900041F09000A6A3E090188375F00924
:103EF80012485DEE75F009A42583F583E4939000DC
:103F080042F090188475F009EF12485DEE75F009DB
:103F1800A42583F583E493900043F09000A6A3E0E2
:103F280090188575F00912485DEE75F009A425838F
:103F3800F583E493FD900044F090188675F009EF3E
:103F480012485DEE75F009A42583F583E49390008B
:103F580045F09000A6A3E090188775F00912485D17
:103F6800EE75F009A42583F583E493900046F0905C
:103F7800188875F009EF12485DEE75F009A42583DD
:103F8800F583E493900047F09000A6A3E090188989
:103F980075F00912485DEE75F009A42583F583E4F0
:103FA80093900048F0ED6015900044E075F010A47F
:103FB80024EFF9741935F0FA7BFF1260F090004590
:103FC800E0FF601175F010A424EFF9741935F0FAC8
:0E3FD8007BFF126121900040E0900000F0227B
:105A7F0090003B7424F090003C7407F0E4900049D0
:105A8F00F090004AF0900039E090004BF07BFF7AE5
:105A9F001A79EF1260F012611B7F0F12449F900072
:105AAF0005E0FF124470900006E0FF1244707F1E65
:0A5ABF0012449F9000007432F022A0
:103FE6001251D9D39000A7E094009000A6E0940067
:103FF600400A1260EA90000074FAF0229000A6E0EF
:10400600FEA3E0FF9018DB75F00912485DEE75F02F
:1040160009A42583F583E493900040F09018DC759D
:10402600F009EF12485DEE75F009A42583F583E4E7
:1040360093900041F09000A6A3E09018DD75F0097A
:1040460012485DEE75F009A42583F583E49390008C
:1040560042F09018DE75F009EF12485DEE75F00932
:10406600A42583F583E493900043F09000A6A3E093
:104076009018DF75F00912485DEE75F009A42583E6
:10408600F583E493FD900044F09018E075F009EF95
:1040960012485DEE75F009A42583F583E49390003C
:1040A60045F09000A6A3E09018E175F00912485D6E
:1040B600EE75F009A42583F583E493900046F0900D
:1040C60018E275F009EF12485DEE75F009A4258334
:1040D600F583E493900047F09000A6A3E09018E3E0
:1040E60075F00912485DEE75F009A42583F583E4A1
:1040F60093900048F0ED6015900044E075F010A430
:10410600240FF9741A35F0FA7BFF1260F09000451F
:10411600E0FF601175F010A4240FF9741A35F0FA57
:0E4126007BFF126121900040E0900000F0222B
:105AC90090003B7429F090003C7407F0E490004981
:105AD900F090004AF090003AE090004BF07BFF7A9A
:105AE9001A79FF1260F012611B7F0D12449F90001A
:105AF90005E0FF124470900006E0FF1244707F1E1B
:0A5B090012449F9000007432F02255
:104134001251D9D39000A7E094009000A6E0940017
:10414400400A1260EA90000074FAF0229000A6E09F
:10415400FEA3E0FF90193575F00912485DEE75F085
:1041640009A42583F583E493900040F090193675F3
:10417400F009EF12485DEE75F009A42583F583E498
:1041840093900041F09000A6A3E090193775F009D0
:1041940012485DEE75F009A42583F583E49390003D
:1041A40042F090193875F009EF12485DEE75F00988
:1041B400A42583F583E493900043F09000A6A3E044
:1041C40090193975F00912485DEE75F009A425833C
:1041D400F583E493FD900044F090193A75F009EFEB
:1041E40012485DEE75F009A42583F583E4939000ED
:1041F40045F09000A6A3E090193B75F00912485DC4
:10420400EE75F009A42583F583E493900046F090BD
:10421400193C75F009EF12485DEE75F009A4258389
:10422400F583E493900047F09000A6A3E090193D35
:1042340075F00912485DEE75F009A42583F583E451
:1042440093900048F0ED6015900044E075F010A4E0
:10425400247FF9741A35F0FA7BFF1260F090004560
:10426400E0FF601175F010A4247FF9741A35F0FA98
:0E4274007BFF126121900040E0900000F022DC
:10617C003049079000007401F02290003B742EF01F
:10618C0090003C7407F07BFF7A1B790F1260F012C1
:0E619C00611B7F1E12449F9000007432F0229F
:105EDA00304F07900000742FF02290000AE06438D7
:105EEA006005A3E0B4390A1260EA90000074FAF07F
:105EFA00227BFF7A1B79BF1260F090000AE0540FF0
:095F0A00F5559000007430F022FE
:105C6F0090000AE064386005A3E0B4390A1260EAD4
:105C7F0090000074FAF0227BFF7A1B791F1260F0FC
:105C8F0090000AE0540FF555D202D20A752EFF127A
:105C9F0033817BFF7A1B79EF1260F090000074FE66
:025CAF00F022E1
:105B130090000AE0540FF555304702D20012339338
:105B2300304719202B04E54470F912338A7BFF7A3E
:105B33001B79EF1260F090000074FEF030481920DA
:105B43002904E54470F912338A7BFF7A1B79EF123B
:095B530060F090000074FEF022E5
:10565200304A56900001E0FF900034F0C24A1244F2
:1056620070900034E0FF1264085021900034E0FF93
:1056720090003CE02403F582E43400F583EFF090DF
:10568200003CE004F0900000E004F022900034E0DE
:10569200B42A079000007403F0227BFF7A1B79CFB3
:0A56A2001260F090000074FAF0228C
:10532C00304A6A900001E0FF900034F0C24A124407
:10533C0070900034E0FFB42A0B90003BE09000002A
:10534C00F0D24F22EFB4230B90003BE0900000F022
:10535C00C24F22900034E0FF1264085021900034B8
:10536C00E0FF90003CE02403F582E43400F583EF89
:10537C00F090003CE004F0900000E004F0227BFF91
:0E538C007A1B79CF1260F090000074FAF022C4
:105C2C00304A3F900001E0FF900034F0124470C203
:105C3C004A900034E0FFB42A0B90003BE090000047
:105C4C00F0D24F22EFB4230B90003BE0900000F019
:105C5C00C24F227BFF7A1B79CF1260F09000007448
:035C6C00FAF02229
:0A58AC00900043E0FF7003304F3816
:1058B60012449F1262A0124EAF8F78900041E052C0
:1058C60078E57860047F3180027F30124470304F73
:1058D60017C24FE5782430900023F090003374010E
:0858E600F090000074F0F022C4
:0F58EE00900046E0FF12449F900000E004F0227B
:105BE800304A40900001E0FF900034F0C24A12446D
:105BF80070900034E0FFB42A079000007403F0228C
:105C0800126408500F900034E090000DF0900000EE
:105C1800E004F0227BFF7A1B79CF1260F09000003D
:045C280074FAF022F8
:105F4C00304A32900001E0FF900034F0C24ABF2A80
:105F5C00079000007403F022900034E0B423079003
:105F6C000000E004F0227BFF7A1B79CF1260F090E6
:065F7C00000074FAF0229F
:1056AC001262A09000AAEEF0A3EFF0124EAF8F782A
:1056BC0090003D7401F090000DE0B4310890004171
:1056CC00E04278800E90000DE0B4301E900041E076
:1056DC00F452789000AAE0FEA3E0FFAD78124E726F
:1056EC001263B390000074FEF0227BFF7A1B79CF1B
:0956FC001260F090000074FAF055
:015705002281
:10516400900043E0FF7003304F5612449F1262A038
:105174009000AAEEF0A3EFF0E4F578900041E0FF90
:10518400E578C39F50279000AAE475F001124847C0
:10519400AFF0FE124EAF8F7974232578F582E43494
:1051A40000F583E579F0124470057880CE304F1015
:1051B400C24FE57804900033F090000074F0F022C0
:1051C40090003C740AF0900046E0FF12449F900067
:0451D40000E004F003
:0151D80022B4
:10507600304A75900001E0FF900034F0C24A1244B5
:1050860070900034E0FFB42A079000007403F02209
:10509600EFB42308900000E004F080391264085051
:1050A60038900034E0FF90003CE0FE04F074032EDC
:1050B600F582E43400F583EFF0900041E02409FF27
:1050C600E433FE90003CE0D39FEE6480F874809851
:1050D6004016900000E004F0227BFF7A1B79CF1285
:0950E60060F090000074FAF02261
:105E9F00304A37900001E0FF900034F0C24A1244BC
:105EAF0070900034E0FFB42A079000007403F022D2
:105EBF00EFB42307900000E004F0227BFF7A1B79F8
:0B5ECF00CF1260F090000074FAF02287
:105760001262A09000AAEEF0A3EFF090003C740A41
:10577000F0E4F578900041E0FFE578C39F50279072
:1057800000AAE475F001124847AFF0FE90003CE03B
:10579000FD04F074032DF582E43400F583E0FD127E
:1057A0004E72057880CE7BFF7A1B79EF1260F09005
:0557B000000074FEF092
:0157B50022D1
:10524E00304A6B900001E0FF900034F0C24A1244E5
:10525E0070900034E0FFB42A079000007403F0222F
:10526E00126408501A900034E0FF90003CE0FE04F7
:10527E00F074032EF582E43400F583EFF080107B9A
:10528E00FF7A1B79CF1260F090000074FAF0229032
:10529E000041E02409FFE433FE90003CE0D39FEE92
:0F52AE006480F87480984006900000E004F022BD
:10488F00900043E0FF7006204F0302493A12449F05
:10489F001262A09000AAEEF0A3EFF0124EAF122C0E
:1048AF0031900041E0B401109000A3E0FF1244707A
:1048BF009000A3E0900023F0900041E0B40220901C
:1048CF0000A2E0FF1244709000A3E0FF124470902A
:1048DF0000A2E0900023F09000A3E0900024F0905D
:1048EF000041E0640370309000A1E0FF124470902B
:1048FF0000A2E0FF1244709000A3E0FF12447090FA
:10490F0000A1E0900023F09000A2E0900024F0902E
:10491F0000A3E0900025F0304F11C24F900041E00E
:10492F00900033F090000074F0F022900046E0FF0A
:10493F0012449F90003C740AF0900000E004F022B3
:1059E900122C875002803B122C5F8F78900047E081
:1059F900FFE578C39F402B900048E0FFE578D39FEF
:105A090050201262A09000AAEEF0A3EFF0AD781238
:105A19004E727BFF7A1B79EF1260F090000074FEE2
:0B5A2900F0221260EA90000074FAF016
:015A3400224F
:1058FD00122C875002803F122C5F8F78900047E06A
:10590D00FFE578C39F400B900048E0FFE578D39FFB
:10591D004004E57870201262A09000AAEEF0A3EF8B
:10592D00F0AD78124E727BFF7A1B79EF1260F0901A
:0F593D00000074FEF0221260EA90000074FAF08D
:01594C002238
:104F7D00900043E0FF7003304F5E12449F1262A019
:104F8D009000AAEEF0A3EFF0124EAF8F78124EF80C
:104F9D00E4F57874A12578F582E43400F583E0FF1B
:104FAD0074232578F582E43400F583EFF074A125A0
:104FBD0078F582E43400F583E0FF1244700578E55E
:104FCD0078C3940440CD304F0FC24F90003374031B
:104FDD00F090000074F0F022900046E0FF12449F24
:0C4FED0090003C740AF0900000E004F01A
:014FF9002295
:105D31007F0A1245EE8F78E57860121262A090001A
:105D4100AAEEF0A3EFF0E57814FD124E72E5787B30
:105D5100FF600E7A1B79EF1260F090000074FEF084
:0E5D6100227A1B796F1260F090000074FAF045
:015D6F002211
:104AC500900043E0FF7006204F03024B6012449FA5
:104AD5001262A09000AAEEF0A3EFF0124EAF122CD6
:104AE500319000AAE475F001124847AFF0FE124E6E
:104AF500AF122C159000A2E0FF900023F0A3F01256
:104B050044709000A3E0FF1244709000AAE475F091
:104B150001124847AFF0FE124EAF122C159000A1BE
:104B2500E0FF900025F09000A2E0900026F09000B4
:104B3500A3E0900027F01244709000A2E0FF124419
:104B4500709000A3E0FF124470304F0FC24F9000E9
:104B5500337405F090000074F0F022900046E0FFF9
:104B650012449F90003C740AF0900000E004F0228B
:10494F0090000DE0540F75F00AA4FFA3E0540F2F51
:10495F00F578900010E0540F75F00AA4FDACF090BC
:10496F00000FE0540F75F064A42DFFE5F03CFE90AE
:10497F000011E0540F7C002FFFEC3EFEE578C3944E
:10498F00014019E578D394145012C3EF9401EE94BB
:10499F00004009D3EF94FAEE9400400A1260EA90B7
:1049AF00000074FAF0221262A09000AAEEF0A3EFBA
:1049BF00F09000AAE475F001124847AFF0FEAD7811
:1049CF00124E72900010E0540F75F00AA4FF900081
:1049DF000FE0540F75F064A42FFF900011E0540FF7
:1049EF002FF5789000AAE0FEA3E0FFAD78124E728B
:0F49FF007BFF7A1B79EF1260F090000074FEF0DE
:014A0E002285
:103955007F0D1245EEEF701A900010E0B43010A301
:10396500E0B4300BA3E0B43006A3E064306003029A
:103975003A4E900014E0FF64306004EFB4350E90C9
:103985000015E0540FD394054003023A4E900014FD
:10399500E0FF64316004EFB43611900019E0B42003
:1039A50007900018E0B42003023A4E900014E0FF9F
:1039B50064326004EFB43711900018E0B42007902A
:1039C5000017E0B42003023A4E900014E0FF643380
:1039D5006004EFB43809900015E0B42002806A90C5
:1039E5000014E0FF64346005EF64397066900015DB
:1039F500E0540F75F00AA4FFA3E0540F2FF578905B
:103A05000018E0540F75F00AA4FDACF0900017E023
:103A1500540F75F064A42DFFE5F03CFE900019E00D
:103A2500540F7C002FFFEC3EFEE578C3940140194E
:103A3500E578D394145012C3EF9401EE9400400935
:103A4500D3EF94FAEE9400400A1260EA90000074F5
:103A5500FAF0221262A09000AAEEF0A3EFF0900017
:103A65003C740AF0E4F578900041E0FFE578C39FE7
:103A750050279000AAE475F001124847AFF0FE9078
:103A8500003CE0FD04F074032DF582E43400F58379
:103A9500E0FD124E72057880CE7BFF7A1B79EF121E
:083AA50060F090000074FEF0D7
:013AAD0022F6
:104FFA00900043E0FF7003304F5B12449F1262A09F
:10500A009000AAEEF0A3EFF0E4F578900041E0FFFB
:10501A00E578C39F502C9000AAE475F00112484726
:10502A00AFF0FE124EAF8F7974232578F582E434FF
:10503A0000F583E579F07E00124EAF1244700578D0
:10504A0080C9304F10C24FE57804900033F09000C9
:10505A000074F0F022900046E0FF12449F90003C5A
:0B506A00740AF0D24D900000E004F04A
:015075002218
:10539A00304A65900001E0FF900034F0C24ABF2A0B
:1053AA00079000007403F022900034E0FFB4230851
:1053BA00900000E004F0803DEF547FFF12447090AB
:1053CA000034E0547FFF90003CE0FE04F074032EAA
:1053DA00F582E43400F583EFF0900041E02409FF00
:1053EA00E433FE90003CE0D39FEE6480F87480982A
:0953FA004006900000E004F022DE
:10594D00304A4B900001E0FF900034F0C24ABF2A6C
:10595D00079000007403F022900034E0FFB4230B95
:10596D00900000E004F0E004F08010126408500F85
:10597D00900034E090003EF0900000E004F0227BB7
:0F598D00FF7A1B79CF1260F090000074FAF022BD
:104C1500204A03024CB1900001E0FF900034F0C23D
:104C25004ABF2A079000007403F022900034E0FF89
:104C3500B4230A900000E004F0E004F022126408B6
:104C4500505B90003EE0540F75F00AA4FF900034CD
:104C5500E0540F2FF0E0901DE893FF900034F01220
:104C65004470900034E0FF90003CE0FE04F07403D3
:104C75002EF582E43400F583EFF0900041E024093D
:104C8500FFE433FE90003CE0D39FEE6480F874802F
:104C950098900000E0400304F02214F0227BFF7A94
:0D4CA5001B79CF1260F090000074FAF0222D
:106252003047099000B5E0F55A122B3B304903E470
:10626200F55A30480B304505755A0A8003755A288D
:07627200900000E004F0229F
:10540300E55A70641246DC900040E0124869543358
:105413006454386E54387854388254388C543D96DA
:105423005442A05447AA544CB45451BE000054549F
:1054330012631E801C12614C80171265A080121229
:1054430065A1800D1265A280081265A38003126511
:10545300A430470E9000B4E07880F6900000E0049A
:09546300F0229000007401F02217
:0F63F9007880E67009122B419000007401F022A9
:1057060030470D9000B5E0F55A122B3BE55A70FC78
:10571600304807755A05E55A70FCE4F57830480CB0
:10572600126507122BE0126587122BE030470C1228
:105736006512122BE0126587122BE00578E578C317
:10574600940540D930470C9000B4E07880F6788014
:09575600E670FB9000007401F004
:01575F002227
:01659C0022DC
:01659D0022DB
:01659E0022DA
:1052BD0030480A2045079000007401F02230470D58
:1052CD009000B5E0F55A122B3BE55A70FC304807BB
:1052DD00755A05E55A70FC304715126512E4F578DC
:1052ED00122BE00578E578C3940A40F412658730F7
:1052FD004815126507E4F578122BE00578E578C3BB
:10530D00940A40F412658730470C9000B4E0788021
:0E531D00F67880E670FB126087E4900000F0E6
:01532B00225F
:01659F0022D9
:105D7000302B3B204A38755B64E54B547FFF90170E
:105D80005393900001F0304D0EE54B30E709EF9052
:105D9000176393900001F0D24AC22B900001E0B447
:0F5DA0002307900002E004F022E4900002F022BA
:105DAF0030293B204A38755B64E549547FFF9017D3
:105DBF005393900001F0304D0EE54930E709EF9015
:105DCF00176393900001F0D24AC229900001E0B40A
:0F5DDF002307900002E004F022E4900002F0227B
:10351B00204B03023688304A03023688900002E0C3
:10352B00F578E4F0755B64126598D24ABF3007906A
:10353B0000017430F022BF31079000017431F0228A
:10354B00BF32079000017432F022BF3307900001A5
:10355B007433F022BF34079000017434F022BF356E
:10356B00079000017435F022BF36079000017436C6
:10357B00F022BF37079000017437F022BF38079055
:10358B0000017438F022BF39079000017439F02222
:10359B00BF23109000017423F0AF780578900002E0
:1035AB00EFF022BF2A07900001742AF022BF4107D7
:1035BB009000017441F022BF42079000017442F069
:1035CB0022BF43079000017443F022BF64079000B1
:1035DB00017444F022204D03C24A22BF61079000C0
:1035EB00017461F022BF62079000017462F022BF88
:1035FB0063079000017463F022BF640790000174AD
:10360B0064F022BF65079000017465F022BF660766
:10361B009000017466F022BF67079000017467F099
:10362B0022BF68079000017468F022BF6907900001
:10363B00017469F022BF6A07900001746AF022BF1F
:10364B006B07900001746BF022BF6C079000017444
:10365B006CF022BF6D07900001746DF022BF6E07F6
:10366B00900001746EF022BF6F07900001746FF031
:0D367B0022BF70079000017470F022C24A57
:01368800221F
:0B64D7007F209000037420F0A3DFFC86
:0164E2002297
:0F640800EFC394304007EFD39439500122C322E1
:1051D90090000CE0FD6420602E90000BE0540F75E8
:1051E900F00AA4FBAAF090000AE0540F75F064A439
:1051F9002BFFE5F03AFEED540F7C002FFFEC3E90BB
:1052090000A6F0A3EF803190000BE0FD6420900030
:105219000A601AE0540F75F00AA4FFED540F7C00E0
:105229002FFEEC35F09000A6F0A3CE800BE0540FD2
:10523900FF9000A6E4F0A3EFF0E024FFF09000A6B1
:05524900E034FFF0223B
:10546C00900009E0FD6420602B900008E0540F755B
:10547C00F00AA4FBAAF0900007E0540F75F064A4A6
:10548C002BFFE5F03AFEED540F7C002FFFEC3E9025
:10549C0000A8802E900008E0FD6420900007601AA0
:1054AC00E0540F75F00AA4FFED540F7C002FFEECB6
:1054BC0035F09000A8F0A3CEF022E0540FFF90003E
:0754CC00A8E4F0A3EFF022B9
:1062C300900005E0540F75F00AA4FFA3E0540F2FCC
:1062D300900035F0D394004006E09415500122C39A
:0162E3002298
:10559900E4FFEF75F003A424FFF582E4341BF583DF
:1055A900E493FE900004E0FDEE6D703BEF75F003AF
:1055B900A42400F582E4341CF583E493FE900005ED
:1055C900E0FDEEB50521EF75F003A42401F582E4B1
:1055D900341CF583E493FE900006E0FDEEB5050763
:0C55E900900036EFF0D3220FBF33A7C3B1
:0155F5002293
:10553900E4FF75F003EFA42498F582E5F0341CF537
:1055490083E493FE900004E0FDEE6D703D75F00379
:10555900EFA42499F582E5F0341CF583E493FE90D9
:105569000005E0FDEEB5052275F003EFA4249AF5D8
:1055790082E5F0341CF583E493FE900006E0FDEE2D
:0F558900B50507900037EFF0D3220FBF70A4C312
:0155980022F0
:1045EE0074032FF582E43400F583E0FD64317069C5
:1045FE00FE74042FF582E43400F583E0FCEE75F0D2
:10460E0003A424FFF582E4341BF583E4936C70421B
:10461E0074052FF582E43400F583E0FCEE75F003AB
:10462E00A42400F582E4341CF583E493B5042374CA
:10463E00062FF582E43400F583E0FCEE75F003A45A
:10464E002401F582E4341CF583E493B50404EE04EE
:10465E00FF220EBE339B7F0022ED6432706DFE741E
:10466E00042FF582E43400F583E0FD75F003EEA42B
:10467E002498F582E5F0341CF583E4936D7045744F
:10468E00052FF582E43400F583E0FD75F003EEA40A
:10469E002499F582E5F0341CF583E493B505257471
:1046AE00062FF582E43400F583E0FD75F003EEA4E9
:1046BE00249AF582E5F0341CF583E493B50505EEF6
:0D46CE002434FF220EBE70977F00227F0073
:0146DB0022BC
:104EF800EFC394339000A150397431F0EF75F0038B
:104F0800A424FFF582E4341BF583E4939000A2F017
:104F1800EF75F003A42400F582E4341CF583E493D0
:104F28009000A3F0EF75F003A42401F582E4341C8B
:104F3800803A7432F075F003EFA424FFF582E5F0AF
:104F4800341BF583E4939000A2F075F003EFA424DA
:104F580000F582E5F0341CF583E4939000A3F07526
:104F6800F003EFA42401F582E5F0341CF583E49303
:054F78009000A4F022EE
:10637400900005E0540F75F00AA4FFA3E0540F2F1A
:05638400900038F0223A
:10638900900005E0540F75F00AA4FFA3E0540F2F05
:05639900900039F02224
:10639E00900005E0540F75F00AA4FFA3E0540F2FF0
:0563AE0090003AF0220E
:0660EA007BFF7A1B793FE9
:0660F0008B798A7A897B9E
:1060F6007F0112449FE4F57CAB79AA7AA97B857C63
:10610600827583001247C5FF124470057CE57CC387
:04611600941040E4BD
:01611A002262
:06611B007BFF7A1B798F67
:066121008B798A7A897B6C
:106127007F1112449FE4F57CAB79AA7AA97B857C21
:10613700827583001247C5FF124470057CE57CC356
:04614700941040E48C
:01614B002231
:1062A00090004BE0FF90004AE08FF0A4FF9000497F
:1062B000E07C002FFFEC35F0FE900042E02FFFEC79
:0362C0003EFE227D
:1063B300900044E075F010A424D3F9741E35F0FA6C
:0563C3007BFF026121D7
:036598007F03225C
:10630300E4F578AF787E00E57890203393FD124E64
:0A631300720578E578C3941040E9A4
:01631D00225D
:105F1300E4F578E4F579E57875F017A42464FFE4F3
:105F230035F0FE7C00EF2579FFEC3EFEE57990200D
:105F33005793FD124E720579E579C3941740D7053F
:085F430078E578C3946440CBBB
:015F4B002233
:10627900E4F578AF787E00124EAF74AC2578F582DC
:10628900E43400F583EFF00578E578C3941040E332
:066299009000ACE0F524CA
:01629F0022DC
:10631E00304708900023E0FF1264EF3048089000E9
:07632E0023E0FF1264E322EB
:10614C00E4F578900033E0FFE578C39F5021742389
:10615C002578F582E43400F583E0F579304704FFC7
:0F616C001264EF304805AF791264E3057880D4F0
:01617B002201
:0165A00022D8
:0165A10022D7
:0165A20022D6
:0165A30022D5
:0165A40022D4
:0C64E300126577122BE012658E022BE090
:0C64EF0012657F122BE012658E022BE07C
:1046DC00E4F578F579F57A9000A7E02401FF9000D5
:1046EC00A6E03400FEC3EF940AEE94005005A3E05C
:1046FC0004F57AD3EF9463EE9400404C9000A7E05D
:10470C002401FB9000A6E03400FA7C007D64AF032A
:10471C00FE1247F28F78EF75F064A4FFC3EB9FFF96
:10472C00EA95F0FE7C007D0A1247F28F79A3E00433
:10473C00FFE57875F064A4FEC3EF9EFFE57975F094
:10474C000AA4FEC3EF9EF57A9000A7E02401FF9027
:10475C0000A6E03400FED3EF9409EE940040197CDF
:10476C00007D0A1247F28F79A3E004FFE57975F01A
:10477C000AA4FEC3EF9EF57A74302578F578743070
:10478C002579F5797430257AF57A304714AF78129B
:10479C0064EFAF791264EFAF7A1264EF7F2A126480
:1047AC00EF304814AF781264E3AF791264E3AF7A58
:0847BC001264E37F2A1264E39A
:0147C40022D2
:1044E60009920A9E0BC70D100E7D101211D213C52C
:1044F60015ED185208D0094E09D40A600AF40B913A
:104506000C360CE50D9D0E600F2D100610EB11DD1F
:1045160012DC13EA15071633177118C01D2107B1EF
:1045260007E808200859196E1A211ADA1B971C5A2F
:104536000894090E09900A190AA90B410BE30C8C81
:104546000D3F0DFD0EC50F9810771162125B1362B9
:104556001477159B16D018161DEF1EC21F9B2079C7
:10456600215F224A233B24342533263912330FCDCB
:1045760014331566169A17CD19000E9A1366110094
:1045860011661033150016331766189A19CD0DCD1E
:104596000F00129A11CD1300149A15CD1700183377
:1045A60019660E330F66109A191823A01296203D2D
:1045B600129623A0129627631488203D148823A000
:1045C6001488276316B8203D16B823A016B82763AB
:1045D6001918203D1918276312962B8C14882B8CDA
:0845E60016B82B8C19182B8C60
:0B65070075081575095ED22DD2032225
:0B65120075081575095ED22DD20B2212
:07658700C22DC203C20B226A
:086577001237F4D22ED20422E7
:08657F001237F4D22ED20C22D7
:0937F400E4F512F513F514F515C6
:1037FD00EF12486938F82338E72A38353038473121
:10380D00385932386B33387D34388F3538A13638E6
:10381D00B33738C53838D639390941391A42392BB9
:10382D0043393C44000039549045AEE493F50D7492
:10383D000193F50E9045B002394B9045B2E493F5E6
:10384D000D740193F50E9045B402394B9045B6E4D5
:10385D0093F50D740193F50E9045B802394B9045D3
:10386D00BAE493F50D740193F50E9045BC02394BF6
:10387D009045BEE493F50D740193F50E9045C0028D
:10388D00394B9045C2E493F50D740193F50E9045B7
:10389D00C402394B9045C6E493F50D740193F50EB2
:1038AD009045C802394B9045CAE493F50D740193C8
:1038BD00F50E9045CC02394B9045CEE493F50D7441
:1038CD000193F50E9045D080759045D2E493F50D9A
:1038DD00740193F50E9045D480649045D6E493F52C
:1038ED000D740193F50E9045D880539045DAE4930D
:1038FD00F50D740193F50E9045DC80429045DEE4A4
:10390D0093F50D740193F50E9045E080319045E2ED
:10391D00E493F50D740193F50E9045E480209045E8
:10392D00E6E493F50D740193F50E9045E8800F9044
:10393D0045EAE493F50D740193F50E9045ECE4938F
:08394D00F50F740193F510223F
:07658E00C22EC20CC2042260
:030000000264FB9C
:0C64FB00787FE4F6D8FD7581B8022DA46E
:1047C500BB010CE58229F582E5833AF583E02250A9
:1047D50006E92582F8E622BBFE06E92582F8E222F3
:0D47E500E58229F582E5833AF583E493220D
:1047F200BC000BBE0029EF8DF084FFADF022E4CCAB
:10480200F875F008EF2FFFEE33FEEC33FCEE9DEC73
:10481200984005FCEE9DFE0FD5F0E9E4CEFD22EDB9
:10482200F8F5F0EE8420D21CFEADF075F008EF2F03
:10483200FFED33FD4007985006D5F0F222C398FDF4
:054842000FD5F0EA2291
:10484700A3F8E0C5F025F0F0E58215827002158324
:06485700E0C838F0E82281
:0C485D00A42582F582E5F03583F5832266
:10486900D083D082F8E4937012740193700DA3A3DE
:1048790093F8740193F5828883E4737402936860F2
:06488900EFA3A3A380DFF2
:00000001FF
